:020000040000FA
:040800004EEF07F0C0
:1008100003B210EF05F0F2B42BEF05F09EB033EF0A
:1008200005F09EB23BEF05F0F2A81AEF04F0F2B229
:1008300025EF04F0F2A620EF04F0F2B022EF04F06E
:100840002CEF07F0F296F290FF00CD90F2929EA06E
:100850002FEF04F00101463F2FEF04F0472BA1C119
:10086000A5F1A2C1A6F1A3C1A7F1A4C1A8F19DC1A0
:10087000A1F19EC1A2F19FC1A3F1A0C1A4F199C1B0
:100880009DF19AC19EF19BC19FF19CC1A0F195C1C0
:1008900099F196C19AF197C19BF198C19CF191C1D0
:1008A00095F192C196F193C197F194C198F18DC1E0
:1008B00091F18EC192F18FC193F190C194F189C1F0
:1008C0008DF18AC18EF18BC18FF18CC190F1CECFA9
:1008D00089F1CFCF8AF146C18BF147C18CF1CF6A44
:1008E000CE6A0101466B476B9E90CD800EBC0E8E8A
:1008F0000EBA7EEF04F00E8A2CEF07F00E8C0EBEBF
:10090000BAEF04F089C18DF18AC18EF18BC18FF1EC
:100910008CC190F18DC191F18EC192F18FC193F193
:1009200090C194F191C195F192C196F193C197F163
:1009300094C198F195C199F196C19AF197C19BF133
:1009400098C19CF199C19DF19AC19EF19BC19FF103
:100950009CC1A0F19DC1A1F19EC1A2F19FC1A3F1D3
:10096000A0C1A4F1A1C1A5F1A2C1A6F1A3C1A7F1A3
:10097000A4C1A8F10101516B526B536B546B8951A7
:1009800051278A5152238B5153238C5154238D511B
:1009900051278E5152238F515323905154239151FB
:1009A00051279251522393515323945154239551DB
:1009B00051279651522397515323985154239951BB
:1009C00051279A5152239B5153239C5154239D519B
:1009D00051279E5152239F515323A0515423A1517B
:1009E0005127A2515223A3515323A4515423A5515B
:1009F0005127A6515223A7515323A8515423D890CD
:100A00005433533352335133D890543353335233D6
:100A10005133D89054335333523351332CEF07F0C2
:100A20000392030103EE00F080517F0BE92604C01E
:100A3000EFFF802B8151805D700BD8A48B8200006A
:100A40008051815D700BD8A48B9281518019D8B4EC
:100A500007902CEF07F0F2940101383F2CEF07F0DC
:100A6000392B2CEF07F09E900101463F2CEF07F049
:100A7000472B2CEF07F09E9204005CA140EF05F09D
:100A8000077C07AC5BEF05F0C274C2B455EF05F00C
:100A9000C3CFADF5C4CFAEF50501D890AE33AD33BD
:100AA000D890AE33AD335CEF05F0C3CF48F1C4CF7F
:100AB00049F15CEF05F0C28207B4C9EF05F03AC115
:100AC0003EF13BC13FF13CC140F13DC141F151C15B
:100AD00055F152C156F153C157F154C158F189C172
:100AE000A9F18AC1AAF18BC1ABF18CC1ACF18DC166
:100AF000ADF18EC1AEF18FC1AFF190C1B0F191C136
:100B0000B1F192C1B2F193C1B3F194C1B4F195C105
:100B1000B5F196C1B6F197C1B7F198C1B8F199C1D5
:100B2000B9F19AC1BAF19BC1BBF19CC1BCF19DC1A5
:100B3000BDF19EC1BEF19FC1BFF1A0C1C0F1A1C175
:100B4000C1F1A2C1C2F1A3C1C3F1A4C1C4F1A5C145
:100B5000C5F1A6C1C6F1A7C1C7F1A8C1C8F1ADC50D
:100B6000AFF5AEC5B0F5AFC5B1F5B0C5B2F5010191
:100B700048514E2749514F23E86A50230D2EC9EFA3
:100B800005F04FC14AF150C14BF14E6B4F6B506BAA
:100B9000078E0201002F2CEF07F03C0E006F0501BD
:100BA0002951000AD8B478EF06F005012951010A4D
:100BB000D8B402EF06F005012951020AD8B443EF78
:100BC00006F005012951030AD8B443EF06F00501E8
:100BD0002951040AD8B443EF06F005012951050A4A
:100BE000D8B443EF06F005012951060AD8B443EF03
:100BF00006F005012951070AD8B443EF06F0296B26
:100C000078EF06F005014D670DEF06F04E670DEF2A
:100C100006F04F670DEF06F0506711EF06F078EF22
:100C200006F051C500F152C501F153C502F154C59A
:100C300003F10101010E046F000E056F000E066F37
:100C4000000E076FB4EC1BF000C151F501C152F565
:100C500002C153F503C154F5006736EF06F0016792
:100C600036EF06F0026736EF06F0036778EF06F01E
:100C70004DC551F54EC552F54FC553F550C554F508
:100C80000E8878EF06F005012A6749EF06F078EF45
:100C900006F00EBE5EEF06F00FA063EF06F0010156
:100CA0003A675AEF06F03B675AEF06F03C675AEF97
:100CB00006F03D675EEF06F063EF06F007AE63EF08
:100CC00006F075EF06F005012B2F78EF06F03C0ECD
:100CD0002B6F2A2F78EF06F00101000E556FE00E02
:100CE000566FA50E576F010E586F05012A6B0E88BF
:100CF000050105015C6B2DB77FEF06F05C810101FA
:100D00007D678AEF06F07E678AEF06F07F678AEFDD
:100D100006F080678EEF06F0BEEF06F081C100F1AD
:100D200082C101F183C102F184C103F10101010E0D
:100D3000046F000E056F000E066F000E076FB4EC17
:100D40001BF000C181F101C182F102C183F103C135
:100D500084F10067B3EF06F00167B3EF06F00267B6
:100D6000B3EF06F00367BEEF06F07DC181F17EC1EF
:100D700082F17FC183F180C184F10E80D57ED5BE22
:100D800069D0D6CF3AF1D7CF3BF138C13CF1E86A10
:100D9000E8CF3DF10F903AC100F13BC101F13CC1F8
:100DA00002F13DC103F101010A0E046F000E056F4F
:100DB000000E066F000E076FB4EC1BF000AF0F8043
:100DC000010147A7F0EF06F00E9A0E9C0E9E01015E
:100DD000000E516F600E526F3D0E536F080E546F30
:100DE00001013ABF00EF07F03B6700EF07F03C67F7
:100DF00000EF07F03D6700EF07F0F28825EF07F0FE
:100E0000F298516B526B536B546B896B8A6B8B6B83
:100E10008C6B8D6B8E6B8F6B906B916B926B936BFE
:100E2000946B956B966B976B986B996B9A6B9B6BAE
:100E30009C6B9D6B9E6B9F6BA06BA16BA26BA36B5E
:100E4000A46BA56BA66BA76BA86BD76AD66A0101CA
:100E5000386B396B2CEF07F002C0E0FF005001C087
:100E6000D8FF1000A6B232EF07F00CC0A9FF0BC0EC
:100E7000A8FFA69EA69CA684F29E550EA76EAA0E5B
:100E8000A76EA682F28EA694A6B244EF07F01200D7
:100E9000A96EA69EA69CA680A8501200076A0E6A9C
:100EA0000F6A0F010D0EC16E860EC06E030EC26E6C
:100EB0000F01280E896E130E926E080E8A6EF30EC5
:100EC000936E8B6A900E946EF18EF19E0D6A010105
:100ED0004E6B4F6B506B4A6B4B6BF29A01013A6B46
:100EE0003B6B3C6B3D6B3E6B3F6B406B416B426BB6
:100EF000436B446B456B386B396BD76AD66A0F010D
:100F0000280ED56EF28A9D90B00ECD6E0101516B08
:100F1000526B536B546B556B566B576B586B596BCD
:100F20005A6B5B6B5C6B466B476BCF6ACE6A0E9AF3
:100F30000E9C0E9E9D80760ECA6E9D8202013C0E16
:100F4000006FCC6A160E48EC07F0E8CF00F1170EE0
:100F500048EC07F0E8CF01F1180E48EC07F0E8CFB5
:100F600002F1190E48EC07F0E8CF03F1010103AFDD
:100F7000D4EF07F0ABEC1CF0160E0C6E00C10BF0BA
:100F800032EC07F0170E0C6E01C10BF032EC07F0DB
:100F9000180E0C6E02C10BF032EC07F0190E0C6E3D
:100FA00003C10BF032EC07F000C17DF101C17EF10D
:100FB00002C17FF103C180F100C181F101C182F161
:100FC00002C183F103C184F11A0E48EC07F0E8CFA7
:100FD00000F11B0E48EC07F0E8CF01F11C0E48ECC5
:100FE00007F0E8CF02F11D0E48EC07F0E8CF03F15F
:100FF000010103AF2AEF08F0ABEC1CF01A0E0C6EE7
:1010000000C10BF032EC07F01B0E0C6E01C10BF0AF
:1010100032EC07F01C0E0C6E02C10BF032EC07F044
:101020001D0E0C6E03C10BF032EC07F01A0E48ECEB
:1010300007F0E8CF00F11B0E48EC07F0E8CF01F114
:101040001C0E48EC07F0E8CF02F11D0E48EC07F04B
:10105000E8CF03F100C185F101C186F102C187F13A
:1010600003C188F1240EAC6E900EAB6E240EAC6EF4
:10107000080EB86E000EB06E1F0EAF6E0401806BCE
:10108000816B0F01900EAB6E0F019D8A0301806B87
:10109000816BA26B8B9278EC1FF0200E48EC07F06E
:1010A000E8CF29F505012951FF0AD8A45FEF08F020
:1010B000296B200E0C6E29C50BF032EC07F00501F0
:1010C000010E2A6F3C0E2B6F250E48EC07F0E8CF7F
:1010D00000F1260E48EC07F0E8CF01F1270E48ECAE
:1010E00007F0E8CF02F1280E48EC07F0E8CF03F153
:1010F000010103AF96EF08F0ABEC1CF0250E0C6E6F
:1011000000C10BF032EC07F0260E0C6E01C10BF0A3
:1011100032EC07F0270E0C6E02C10BF032EC07F038
:10112000280E0C6E03C10BF032EC07F000C14DF538
:1011300001C14EF502C14FF503C150F500C151F593
:1011400001C152F502C153F503C154F5290E48EC13
:1011500007F0E8CF55F505015651555DD8A055C5A6
:1011600056F505012951020A0EE181B8C3EF08F0D6
:101170000501562FC0EF08F055C556F5C3EF08F02E
:1011800081BA97EF22F0210E48EC07F0E8CF00F18A
:10119000220E48EC07F0E8CF01F1230E48EC07F0EF
:1011A000E8CF02F1240E48EC07F0E8CF03F101018B
:1011B00003AF09EF09F0ABEC1CF0210E0C6E00C17F
:1011C0000BF032EC07F0220E0C6E01C10BF032EC8A
:1011D00007F0230E0C6E02C10BF032EC07F0240E68
:1011E0000C6E03C10BF032EC07F0210E48EC07F057
:1011F000E8CF00F1220E48EC07F0E8CF01F1230E12
:1012000048EC07F0E8CF02F1240E48EC07F0E8CFF5
:1012100003F100C157F501C158F502C159F503C1E9
:101220005AF506EC1FF0C8EC1DF018EC1DF0050196
:101230002951030A12E005012951040A1DE00501A4
:101240002951050A24E005012951060A32E0050169
:101250002951070A38E06CEF09F0A6C500F1010139
:101260000F0E001701010051000A36E00101005184
:10127000050A32E069EF09F0A6C500F101010F0E81
:10128000001701010051000A27E069EF09F005018C
:10129000A651000A21E00501A651150A1DE005012D
:1012A000A651300A19E00501A651450A15E069EF7B
:1012B00009F00501A651000A0FE00501A651300A08
:1012C0000BE069EF09F00501A651000A05E069EF9E
:1012D00009F081BA97EF22F007900001F28EF28CAC
:1012E00007B04CEF19F00EB02DEF14F00EB81FEF51
:1012F0000EF00301805181197F0BD8B44CEF19F027
:1013000013EE00F081517F0BE126812BE7CFE8FF40
:10131000E00BD8B44CEF19F023EE82F0A2511F0B72
:10132000D926E7CFDFFFA22BDF50780AD8A44CEFF5
:1013300019F0078081C100F182C101F183C102F17E
:1013400084C103F10101040E046F000E056F000E4D
:10135000066F000E076FB4EC1BF000AFB9EF09F099
:101360000101030E816F000E826F000E836F000E6D
:10137000846F03018251720AD8B42DEF14F08251A8
:10138000520AD8B42DEF14F08251750AD8B42DEF5B
:1013900014F08251630AD8B408EF16F08251690A3A
:1013A000D8B4E8EF10F082517A0AD8B4FBEF11F00C
:1013B0008251490AD8B487EF10F08251500AD8B44C
:1013C000A5EF0FF08251700AD8B4E8EF0FF0825108
:1013D000540AD8B413EF10F08251740AD8B459EFFC
:1013E00010F08251730AD8B45DEF13F08251530AA2
:1013F000D8B4C2EF13F082514C0AD8B415EF0AF0FA
:101400003DEF16F0040114EE00F080517F0BE12651
:1014100082C4E7FF802B12000D0E826F02EC0AF0EF
:101420000A0E826F02EC0AF0120003018351300AA7
:10143000D8B4ACEF0CF003018351310AD8B4FAEF01
:101440000CF003018351320AD8B44AEF0DF00301C6
:101450008351330AD8B44EEF0DF003018351340A9F
:10146000D8B45CEF0DF003018351350AD8B424EFF2
:101470000EF0030183514D0AD8B425EF0BF00301A0
:1014800083516D0AD8B43FEF0BF003018351490A31
:10149000D8B424EF0FF003018351500AD8B456EFAB
:1014A0000EF003018351540AD8B4CFEF0EF00301BC
:1014B0008351630AD8B45FEF0BF003018351430AF1
:1014C000D8B457EF0CF003018351730AD8B45DEF21
:1014D0000BF003018351610AD8B472EF0AF0D8A46B
:1014E0003DEF16F004014C0E826F02EC0AF004018D
:1014F000610E826F02EC0AF0C8EC1DF004012C0EA4
:10150000826F02EC0AF0ABEC1CF0A5C500F1010102
:101510004EEC1CF025C182F40401300E822702EC4F
:101520000AF026C182F40401300E822702EC0AF090
:1015300027C182F40401300E822702EC0AF0040174
:101540002C0E826F02EC0AF0ABEC1CF0A6C500F189
:1015500001014EEC1CF025C182F40401300E8227FB
:1015600002EC0AF026C182F40401300E822702EC5C
:101570000AF027C182F40401300E822702EC0AF03F
:1015800004012C0E826F02EC0AF0ABEC1CF0A7C534
:1015900000F101014EEC1CF025C182F40401300E73
:1015A000822702EC0AF026C182F40401300E822761
:1015B00002EC0AF027C182F40401300E822702EC0B
:1015C0000AF004012C0E826F02EC0AF0ABEC1CF066
:1015D000A8C500F101014EEC1CF025C182F4040104
:1015E000300E822702EC0AF026C182F40401300E8C
:1015F000822702EC0AF027C182F40401300E822710
:1016000002EC0AF004012C0E826F02EC0AF0ABEC43
:101610001CF0ADC500F101014EEC1CF025C182F4B7
:101620000401300E822702EC0AF026C182F4040184
:10163000300E822702EC0AF027C182F40401300E3A
:10164000822702EC0AF052EF0EF0ECEC1CF084C39F
:1016500027F1F9EC1CF070EC1CF0200E0C6E00C1B0
:101660000BF032EC07F000C129F505012951000A01
:1016700006E005012951010A02E06EEC1EF00401AA
:101680004C0E826F02EC0AF004014D0E826F02ECE8
:101690000AF004012C0E826F02EC0AF0ABEC1CF095
:1016A00029C500F14EEC1CF027C182F40401300E74
:1016B000822702EC0AF052EF0EF097EF22F00401BD
:1016C0004C0E826F02EC0AF00401630E826F02EC92
:1016D0000AF018EC1DF004012C0E826F02EC0AF0E7
:1016E00074EC0BF052EF0EF0ABEC1CF0ABC500F15C
:1016F0000101003B0F0E00174EEC1CF027C182F4D5
:101700000401300E822702EC0AF0ABC500F10101A2
:101710000F0E010100174EEC1CF027C182F40401EA
:10172000300E822702EC0AF004012D0E826F02ECCB
:101730000AF0AAC500F10101003B0F0E00174EECA4
:101740001CF027C182F40401300E822702EC0AF05B
:10175000AAC500F101010F0E010100174EEC1CF0AB
:1017600027C182F40401300E822702EC0AF0040142
:101770002D0E826F02EC0AF0A9C500F10101003BB9
:101780000F0E00174EEC1CF027C182F40401300E3E
:10179000822702EC0AF0A9C500F101010F0E010138
:1017A00000174EEC1CF027C182F40401300E822792
:1017B00002EC0AF00401200E826F02EC0AF0A8C5C8
:1017C00000F10F0E010100174EEC1CF027C182F44E
:1017D0000401300E822702EC0AF00401200E826F11
:1017E00002EC0AF0A7C500F101010101003B0F0E58
:1017F00000174EEC1CF027C182F40401300E822742
:1018000002EC0AF0A7C500F101010F0E010100175B
:101810004EEC1CF027C182F40401300E822702EC4A
:101820000AF004013A0E826F02EC0AF0A6C500F13C
:101830000101003B0F0E00174EEC1CF027C182F493
:101840000401300E822702EC0AF0A6C500F1010166
:101850000F0E010100174EEC1CF027C182F40401A9
:10186000300E822702EC0AF004013A0E826F02EC7D
:101870000AF0A5C500F10101003B0F0E00174EEC68
:101880001CF027C182F40401300E822702EC0AF01A
:10189000A5C500F101010F0E00174EEC1CF027C189
:1018A00082F40401300E822702EC0AF0120084C395
:1018B000E8FF0F0BE83AE8CFABF585C3E8FF0F0B65
:1018C0000501AB1387C3E8FF0F0BE83AE8CFAAF591
:1018D00088C3E8FF0F0B0501AA138AC3E8FF0F0BAB
:1018E000E83AE8CFA9F58BC3E8FF0F0B0501A91370
:1018F0008DC3E8FF0F0BE8CFA8F58FC3E8FF0F0BF0
:10190000E83AE8CFA7F590C3E8FF0F0B0501A7134E
:1019100092C3E8FF0F0BE83AE8CFA6F593C3E8FFC0
:101920000F0B0501A61395C3E8FF0F0BE83AE8CFAC
:10193000A5F596C3E8FF0F0B0501A51377EC1DF085
:1019400004014C0E826F02EC0AF00401430E826F18
:1019500002EC0AF069EF0BF058EC22F0ABEC1CF053
:101960002DC500F14EEC1CF004014C0E826F02EC10
:101970000AF00401300E826F02EC0AF004012C0E12
:10198000826F02EC0AF025C182F40401300E822736
:1019900002EC0AF026C182F40401300E822702EC28
:1019A0000AF027C182F40401300E822702EC0AF00B
:1019B00004012C0E826F02EC0AF0ABEC1CF02EC579
:1019C00000F14EEC1CF025C182F40401300E822798
:1019D00002EC0AF026C182F40401300E822702ECE8
:1019E0000AF027C182F40401300E822702EC0AF0CB
:1019F00052EF0EF004014C0E826F02EC0AF004016B
:101A0000310E826F02EC0AF004012C0E826F02ECA0
:101A10000AF025C500F126C501F127C502F128C548
:101A200003F10101100E046F000E056F000E066F2A
:101A3000000E076FE2EC1BF04EEC1CF022C182F4AA
:101A40000401300E822702EC0AF023C182F4040163
:101A5000300E822702EC0AF024C182F40401300E19
:101A6000822702EC0AF025C182F40401300E82279D
:101A700002EC0AF026C182F40401300E822702EC47
:101A80000AF027C182F40401300E822702EC0AF02A
:101A900052EF0EF0C2EC1FF03DEF16F004014C0EB9
:101AA000826F02EC0AF00401330E826F02EC0AF03E
:101AB000F8EC1FF004EF0DF004014C0E826F02EC05
:101AC0000AF00401340E826F02EC0AF004012C0EBD
:101AD000826F02EC0AF0ECEC1CF084C31EF185C3AB
:101AE0001FF186C320F187C321F188C322F189C386
:101AF00023F18AC324F18BC325F18CC326F18DC356
:101B000027F101011D6BF9EC1CF070EC1CF0100EBC
:101B1000046F000E056F000E066F000E076FC3EC1A
:101B20001BF000C121F501C122F502C123F503C15B
:101B300024F50BEC22F02EC5A5F52FC5A6F530C572
:101B4000A7F531C5A8F532C5A9F533C5AAF534C541
:101B5000ABF574EC0BF004012C0E826F02EC0AF072
:101B600035C500F136C501F137C502F138C503F1BD
:101B70000101000E046F000E056F010E066F000ECE
:101B8000076FE2EC1BF04EEC1CF01D67CAEF0DF086
:101B9000CFEF0DF004012D0E826F02EC0AF024C18C
:101BA00082F40401300E822702EC0AF025C182F48F
:101BB0000401300E822702EC0AF004012E0E826F1F
:101BC00002EC0AF026C182F40401300E822702ECF6
:101BD0000AF027C182F40401300E822702EC0AF0D9
:101BE00004012C0E826F02EC0AF0ABEC1CF039C53C
:101BF00000F13AC501F167EC17F004012C0E826F79
:101C000002EC0AF0ABEC1CF03BC500F14EEC1CF012
:101C100025C182F40401300E822702EC0AF026C1AD
:101C200082F40401300E822702EC0AF027C182F40C
:101C30000401300E822702EC0AF052EF0EF00E98EB
:101C4000F8EC1FF052EF0EF004014C0E826F02EC24
:101C50000AF00401350E826F02EC0AF004012C0E2A
:101C6000826F02EC0AF0ABEC1CF00784AFC500F108
:101C700007944EEC1CF025C182F40401300E82273B
:101C800002EC0AF026C182F40401300E822702EC35
:101C90000AF027C182F40401300E822702EC0AF018
:101CA00052EF0EF00CEC0AF03DEF16F004014C0E72
:101CB000826F02EC0AF00401500E826F02EC0AF00F
:101CC00004012C0E826F02EC0AF085C31EF186C35C
:101CD0001FF187C320F188C321F189C322F18AC390
:101CE00023F18BC324F18CC325F18DC326F18EC360
:101CF00027F10101F9EC1CF070EC1CF00301845198
:101D0000530A0DE0030184514D0A38E00401780EB6
:101D1000826F02EC0AF00CEC0AF03DEF16F00401C1
:101D2000530E826F02EC0AF0250E0C6E00C10BF010
:101D300032EC07F0260E0C6E01C10BF032EC07F00E
:101D4000270E0C6E02C10BF032EC07F0280E0C6E61
:101D500003C10BF032EC07F000C14DF501C14EF5A7
:101D600002C14FF503C150F500C151F501C152F553
:101D700002C153F503C154F533EF0FF004014D0ECA
:101D8000826F02EC0AF0290E0C6E00C10BF032ECEF
:101D900007F000C155F500C156F533EF0FF004010F
:101DA0004C0E826F02EC0AF00401540E826F02ECBA
:101DB0000AF004012C0E826F02EC0AF084C31EF1BB
:101DC00085C31FF186C320F187C321F188C322F1A7
:101DD00089C323F18AC324F18BC325F18DC326F176
:101DE0008EC327F10101F9EC1CF070EC1CF001012D
:101DF000000E046F000E056F010E066F000E076FD8
:101E0000C3EC1BF0210E0C6E00C10BF032EC07F09E
:101E1000220E0C6E01C10BF032EC07F0230E0C6E9B
:101E200002C10BF032EC07F0240E0C6E03C10BF074
:101E300032EC07F000C157F501C158F502C159F560
:101E400003C15AF533EF0FF004014C0E826F02EC20
:101E50000AF00401490E826F02EC0AF004012C0E14
:101E6000826F02EC0AF0250E48EC07F0E8CF00F193
:101E7000260E48EC07F0E8CF01F1270E48EC07F0FA
:101E8000E8CF02F1280E48EC07F0E8CF03F14EEC62
:101E90001CF07AEC1AF00401730E826F02EC0AF067
:101EA00004012C0E826F02EC0AF0ABEC1CF0290E40
:101EB00048EC07F0E8CF00F14EEC1CF07AEC1AF099
:101EC0000401730E826F02EC0AF004012C0E826F83
:101ED00002EC0AF051C500F152C501F153C502F1FF
:101EE00054C503F14EEC1CF07AEC1AF00401730EA9
:101EF000826F02EC0AF004012C0E826F02EC0AF0F1
:101F0000ABEC1CF056C500F14EEC1CF07AEC1AF06C
:101F100004016D0E826F02EC0AF004012C0E826F38
:101F200002EC0AF057C500F158C501F159C502F19C
:101F30005AC503F158EC16F004012C0E826F02EC26
:101F40000AF00CEC0AF03DEF16F083C31EF184C3D7
:101F50001FF185C320F186C321F187C322F188C315
:101F600023F189C324F18AC325F18BC326F18CC3E5
:101F700027F10101F9EC1CF070EC1CF0160E0C6E50
:101F800000C10BF032EC07F0170E0C6E01C10BF024
:101F900032EC07F0180E0C6E02C10BF032EC07F0B9
:101FA000190E0C6E03C10BF032EC07F000C17DF18D
:101FB00001C17EF102C17FF103C180F100C181F155
:101FC00001C182F102C183F103C184F187EF10F0F6
:101FD00083C31EF184C31FF185C320F186C321F1A1
:101FE00087C322F188C323F189C324F18AC325F171
:101FF0008BC326F18CC327F10101F9EC1CF070ECC6
:102000001CF000C17DF101C17EF102C17FF103C16D
:1020100080F100C181F101C182F102C183F103C1EC
:1020200084F187EF10F083C31EF184C31FF185C3D1
:1020300020F186C321F187C322F188C323F189C32C
:1020400024F18AC325F18CC326F18DC327F1010148
:10205000F9EC1CF070EC1CF00101000E046F000E96
:10206000056F010E066F000E076FC3EC1BF01A0E12
:102070000C6E00C10BF032EC07F01B0E0C6E01C1B0
:102080000BF032EC07F01C0E0C6E02C10BF032ECC0
:1020900007F01D0E0C6E03C10BF032EC07F000C10F
:1020A00085F101C186F102C187F103C188F187EF93
:1020B00010F083C31EF184C31FF185C320F186C3D2
:1020C00021F187C322F188C323F189C324F18AC394
:1020D00025F18CC326F18DC327F10101F9EC1CF029
:1020E00070EC1CF00101000E046F000E056F010E74
:1020F000066F000E076FC3EC1BF000C185F101C134
:1021000086F102C187F103C188F187EF10F0160E46
:1021100048EC07F0E8CF00F1170E48EC07F0E8CFE5
:1021200001F1180E48EC07F0E8CF02F1190E48EC67
:1021300007F0E8CF03F14EEC1CF07AEC1AF0040142
:10214000730E826F02EC0AF004012C0E826F02EC17
:102150000AF07DC100F17EC101F17FC102F180C1B1
:1021600003F14EEC1CF07AEC1AF00401730E826F4E
:1021700002EC0AF004012C0E826F02EC0AF01A0E37
:1021800048EC07F0E8CF00F11B0E48EC07F0E8CF71
:1021900001F11C0E48EC07F0E8CF02F11D0E48ECEF
:1021A00007F0E8CF03F158EC16F004012C0E826F13
:1021B00002EC0AF085C100F186C101F187C102F18C
:1021C00088C103F158EC16F00CEC0AF03DEF16F064
:1021D0000401690E826F02EC0AF004012C0E826F7A
:1021E00002EC0AF00101040E006F000E016F000EF8
:1021F000026F000E036F4EEC1CF020C182F404014C
:10220000300E822702EC0AF021C182F40401300E64
:10221000822702EC0AF022C182F40401300E8227E8
:1022200002EC0AF023C182F40401300E822702EC92
:102230000AF024C182F40401300E822702EC0AF075
:1022400025C182F40401300E822702EC0AF026C177
:1022500082F40401300E822702EC0AF027C182F4D6
:102260000401300E822702EC0AF004012C0E826F6A
:1022700002EC0AF00101060E006F000E016F000E65
:10228000026F000E036F4EEC1CF020C182F40401BB
:10229000300E822702EC0AF021C182F40401300ED4
:1022A000822702EC0AF022C182F40401300E822758
:1022B00002EC0AF023C182F40401300E822702EC02
:1022C0000AF024C182F40401300E822702EC0AF0E5
:1022D00025C182F40401300E822702EC0AF026C1E7
:1022E00082F40401300E822702EC0AF027C182F446
:1022F0000401300E822702EC0AF004012C0E826FDA
:1023000002EC0AF00101180E006F000E016F000EC2
:10231000026F000E036F4EEC1CF020C182F404012A
:10232000300E822702EC0AF021C182F40401300E43
:10233000822702EC0AF022C182F40401300E8227C7
:1023400002EC0AF023C182F40401300E822702EC71
:102350000AF024C182F40401300E822702EC0AF054
:1023600025C182F40401300E822702EC0AF026C156
:1023700082F40401300E822702EC0AF027C182F4B5
:102380000401300E822702EC0AF004012C0E826F49
:1023900002EC0AF0200EF86EF76AF66A04010900F2
:1023A000F5CF82F402EC0AF00900F5CF82F402ECDA
:1023B0000AF00900F5CF82F402EC0AF00900F5CF2B
:1023C00082F402EC0AF00900F5CF82F402EC0AF084
:1023D0000900F5CF82F402EC0AF00900F5CF82F48F
:1023E00002EC0AF00900F5CF82F402EC0AF00CECE2
:1023F0000AF03DEF16F08351630AD8A43DEF16F0C2
:102400008451610AD8A43DEF16F085516C0AD8A416
:102410003DEF16F08651410A42E08651440A1BE026
:102420008651420AD8B462EF12F08651350AD8B408
:10243000C7EF17F08651360AD8B41CEF18F0865152
:10244000370AD8B485EF18F08651380AD8B4E3EFCC
:1024500018F03DEF16F00798079A04017A0E826F84
:1024600002EC0AF00401780E826F02EC0AF004011B
:10247000640E826F02EC0AF081A846EF12F00401AC
:10248000550E826F02EC0AF04BEF12F004014C0E75
:10249000826F02EC0AF00CEC0AF03DEF16F00788B0
:1024A000079A04017A0E826F02EC0AF00401410ED1
:1024B000826F02EC0AF00401610E826F02EC0AF0F6
:1024C0003CEF12F00798078A04017A0E826F02EC43
:1024D0000AF00401420E826F02EC0AF00401610E60
:1024E000826F02EC0AF03CEF12F00101596780EFB5
:1024F00012F05A6780EF12F05B6780EF12F05C67B2
:1025000098EF12F042678CEF12F043678CEF12F0F5
:1025100044678CEF12F0456798EF12F00101000E4E
:10252000006F000E016F000E026F000E036F1200AD
:102530000101620E046F010E056F000E066F000EA2
:10254000076F59C100F15AC101F15BC102F15CC1D1
:1025500003F1B4EC1BF003BF1CEF13F00101000EFC
:10256000046FA80E056F550E066F020E076F59C156
:1025700000F15AC101F15BC102F15CC103F159C123
:1025800079F15AC17AF15BC17BF15CC17CF1B4ECA9
:102590001BF003BFD5EF12F00101000E796FA80EFA
:1025A0007A6F550E7B6F020E7C6F0E0E48EC07F0B3
:1025B000E8CF0CF10F0E48EC07F0E8CF0DF1100E4C
:1025C00048EC07F0E8CF0EF1110E48EC07F0E8CF29
:1025D0000FF1FDEC1AF079C104F17AC105F17BC16C
:1025E00006F17CC107F1B4EC1BF00782C1EC1AF0D4
:1025F000FDEC1AF00792C1EC1AF079C100F17AC132
:1026000001F17BC102F17CC103F10792C1EC1AF028
:10261000CC0E046FE00E056F870E066F050E076F78
:10262000B4EC1BF000C10CF101C10DF102C10EF1BF
:1026300003C10FF154EF13F00101800E006F1A0E69
:10264000016F060E026F000E036F42C104F143C119
:1026500005F144C106F145C107F1B4EC1BF003AF2D
:1026600035EF13F0ABEC1CF012000E0E48EC07F047
:10267000E8CF0CF10F0E48EC07F0E8CF0DF1100E8B
:1026800048EC07F0E8CF0EF1110E48EC07F0E8CF68
:102690000FF142C100F143C101F144C102F145C152
:1026A00003F10782C1EC1AF00CC100F10DC101F178
:1026B0000EC102F10FC103F112000401730E826F0B
:1026C00002EC0AF004012C0E826F02EC0AF007847F
:1026D00055C159F156C15AF157C15BF158C15CF16E
:1026E0003EC142F13FC143F140C144F141C145F116
:1026F0004AC14CF14BC14DF1079483EC13F00CEC43
:102700000AF03DEF16F059C100F15AC101F15BC169
:1027100002F15CC103F101014EEC1CF07AEC1AF0FD
:102720000401630E826F02EC0AF004012C0E826F2A
:1027300002EC0AF042C100F143C101F144C102F1CF
:1027400045C103F101014EEC1CF07AEC1AF00401D2
:10275000660E826F02EC0AF004012C0E826F02EC0E
:102760000AF0ABEC1CF04CC100F14DC101F10101CC
:102770004EEC1CF07AEC1AF00401740E826F02EC3D
:102780000AF012000F820401530E826F02EC0AF06D
:1027900004012C0E826F02EC0AF083C31EF184C385
:1027A0001FF185C320F186C321F187C322F188C3BD
:1027B00023F189C324F18AC325F18BC326F18CC38D
:1027C00027F10101F9EC1CF070EC1CF000C159F18B
:1027D00001C15AF102C15BF103C15CF18EC31EF16C
:1027E0008FC31FF190C320F191C321F192C322F155
:1027F00093C323F194C324F195C325F196C326F125
:1028000097C327F10101F9EC1CF070EC1CF000C13A
:1028100042F101C143F102C144F103C145F1ECECC5
:102820001CF099C323F19AC324F19BC325F19CC3E7
:1028300026F19DC327F10101F9EC1CF070EC1CF0AE
:1028400000C14CF101C14DF183EC13F004012C0ED9
:10285000826F02EC0AF034EF14F08251520A03E165
:102860000E8234EF14F00E928251750A03E10F8448
:102870003BEF14F00F948251550A03E10F8642EFAB
:1028800014F00F9607840FB29FEF14F00FA48BEF94
:1028900014F0A9C159F1AAC15AF1ABC15BF1ACC1A5
:1028A0005CF1ADC15DF1AEC15EF1AFC15FF1B0C130
:1028B00060F1B1C161F1B2C162F1B3C163F1B4C100
:1028C00064F1B5C165F1B6C166F1B7C167F1B8C1D0
:1028D00068F1B9C169F1BAC16AF1BBC16BF1BCC1A0
:1028E0006CF1BDC16DF1BEC16EF1BFC16FF1C0C170
:1028F00070F1C1C171F1C2C172F1C3C173F1C4C140
:1029000074F1C5C175F1C6C176F1C7C177F1C8C10F
:1029100078F193EF14F055C159F156C15AF157C1EE
:102920005BF158C15CF13EC142F13FC143F140C18E
:1029300044F141C145F14AC14CF14BC14DF10794FD
:102940000EA0C1EF14F001018567AEEF14F08667A9
:10295000AEEF14F08767AEEF14F08867B2EF14F0B3
:10296000C1EF14F075EC12F085C104F186C105F1D8
:1029700087C106F188C107F1B4EC1BF003BF05EF76
:1029800016F075EC12F00101000E046F000E056FD9
:10299000010E066F000E076FE2EC1BF00FA4D8EFDC
:1029A00014F00401750E826F02EC0AF0DDEF14F0F2
:1029B0000401720E826F02EC0AF004012C0E826F89
:1029C00002EC0AF04EEC1CF01D67ECEF14F0040171
:1029D000200E826FEFEF14F004012D0E826F02ECD7
:1029E0000AF024C182F40401300E822702EC0AF0BE
:1029F00025C182F40401300E822702EC0AF00401A2
:102A00002E0E826F02EC0AF026C182F40401300E11
:102A1000822702EC0AF027C182F40401300E8227DB
:102A200002EC0AF004016D0E826F02EC0AF0040160
:102A30002C0E826F02EC0AF042C100F143C101F199
:102A400044C102F145C103F101014EEC1CF07AECE6
:102A50001AF00401480E826F02EC0AF004017A0EAB
:102A6000826F02EC0AF004012C0E826F02EC0AF075
:102A700059C100F15AC101F15BC102F15CC103F11E
:102A800001014EEC1CF07AEC1AF00401630E826F27
:102A900002EC0AF004012C0E826F02EC0AF059C11C
:102AA00000F15AC101F15BC102F15CC103F1010106
:102AB0000A0E046F000E056F000E066F000E076F02
:102AC000C3EC1BF0000E046F120E056F000E066FB4
:102AD000000E076FE2EC1BF04EEC1CF01EC182F4FE
:102AE0000401300E822702EC0AF01FC182F40401B7
:102AF000300E822702EC0AF020C182F40401300E6D
:102B0000822702EC0AF021C182F40401300E8227F0
:102B100002EC0AF022C182F40401300E822702EC9A
:102B20000AF023C182F40401300E822702EC0AF07D
:102B300024C182F40401300E822702EC0AF0040161
:102B40002E0E826F02EC0AF025C182F40401300ED1
:102B5000822702EC0AF026C182F40401300E82279B
:102B600002EC0AF027C182F40401300E822702EC45
:102B70000AF00401730E826F02EC0AF004012C0EBD
:102B8000826F02EC0AF0ABEC1CF04CC100F14DC1BD
:102B900001F167EC17F00EB2D1EF15F00EA003EFC4
:102BA00016F004012C0E826F02EC0AF0200EF86E73
:102BB000F76AF66A04010900F5CF82F402EC0AF024
:102BC0000900F5CF82F402EC0AF00900F5CF82F497
:102BD00002EC0AF00900F5CF82F402EC0AF00900D9
:102BE000F5CF82F402EC0AF00900F5CF82F402EC92
:102BF0000AF00900F5CF82F402EC0AF00900F5CFE3
:102C000082F402EC0AF00CEC0AF00E903DEF16F0A4
:102C10000401630E826F02EC0AF004012C0E826F35
:102C200002EC0AF043EC16F004012C0E826F02EC69
:102C30000AF0B6EC16F004012C0E826F02EC0AF0DA
:102C400032EC17F004012C0E826F02EC0AF0010145
:102C5000F80E006FCD0E016F660E026F030E036F4C
:102C600058EC16F004012C0E826F02EC0AF048ECCE
:102C700017F00CEC0AF03DEF16F00301A26B079081
:102C80000F924CEF19F0D8900E0E48EC07F0E8CFF9
:102C900000F10F0E48EC07F0E8CF01F1100E48EC00
:102CA00007F0E8CF02F1110E48EC07F0E8CF03F18E
:102CB0000101000E046F000E056F010E066F000E7D
:102CC000076FE2EC1BF04EEC1CF01EC182F4040115
:102CD000300E822702EC0AF01FC182F40401300E8C
:102CE000822702EC0AF020C182F40401300E822710
:102CF00002EC0AF021C182F40401300E822702ECBA
:102D00000AF022C182F40401300E822702EC0AF09C
:102D100023C182F40401300E822702EC0AF024C1A0
:102D200082F40401300E822702EC0AF025C182F4FD
:102D30000401300E822702EC0AF004012E0E826F8D
:102D400002EC0AF026C182F40401300E822702EC64
:102D50000AF027C182F40401300E822702EC0AF047
:102D600004016D0E826F02EC0AF01200120E48ECA4
:102D700007F0E8CF00F1130E48EC07F0E8CF01F1BF
:102D8000140E48EC07F0E8CF02F1150E48EC07F0FE
:102D9000E8CF03F101010A0E046F000E056F000E6B
:102DA000066F000E076FC3EC1BF0000E046F120ECF
:102DB000056F000E066F000E076FE2EC1BF04EEC85
:102DC0001CF01EC182F40401300E822702EC0AF0CE
:102DD0001FC182F40401300E822702EC0AF020C1E8
:102DE00082F40401300E822702EC0AF021C182F441
:102DF0000401300E822702EC0AF022C182F40401A1
:102E0000300E822702EC0AF023C182F40401300E56
:102E1000822702EC0AF024C182F40401300E8227DA
:102E200002EC0AF004012E0E826F02EC0AF025C1BA
:102E300082F40401300E822702EC0AF026C182F4EB
:102E40000401300E822702EC0AF027C182F404014B
:102E5000300E822702EC0AF00401730E826F02EC3E
:102E60000AF012000A0E48EC07F0E8CF00F10B0E52
:102E700048EC07F0E8CF01F10C0E48EC07F0E8CF82
:102E800002F10D0E48EC07F0E8CF03F167EF17F001
:102E9000060E48EC07F0E8CF00F1070E48EC07F00B
:102EA000E8CF01F1080E48EC07F0E8CF02F1090E77
:102EB00048EC07F0E8CF03F167EF17F00101ABEC46
:102EC0001CF007844AC100F14BC101F107940101D4
:102ED000E80E046F800E056F000E066F000E076F80
:102EE000C3EC1BF0000E046F040E056F000E066F9E
:102EF000000E076FE2EC1BF0880E046F130E056FD7
:102F0000000E066F000E076FB4EC1BF00A0E046F84
:102F1000000E056F000E066F000E076FE2EC1BF04F
:102F20004EEC1CF001011D679BEF17F00401200E11
:102F3000826F9EEF17F004012D0E826F02EC0AF0F3
:102F400024C182F40401300E822702EC0AF025C16C
:102F500082F40401300E822702EC0AF026C182F4CA
:102F60000401300E822702EC0AF004012E0E826F5B
:102F700002EC0AF027C182F40401300E822702EC31
:102F80000AF00401430E826F02EC0AF0120087C3BC
:102F90001EF188C31FF189C320F18AC321F18BC3BD
:102FA00022F18CC323F18DC324F18EC325F190C38C
:102FB00026F191C327F101011D6BF9EC1CF070ECB7
:102FC0001CF00101000E046F000E056F010E066F6C
:102FD000000E076FC3EC1BF00E0E0C6E00C10BF061
:102FE00032EC07F00F0E0C6E01C10BF032EC07F063
:102FF000100E0C6E02C10BF032EC07F0110E0C6ECD
:1030000003C10BF032EC07F004017A0E826F02EC80
:103010000AF004012C0E826F02EC0AF00401350E56
:10302000826F02EC0AF004012C0E826F02EC0AF0AF
:1030300043EC16F04BEF12F087C31EF188C31FF16B
:1030400089C320F18AC321F18BC322F18CC323F100
:103050008DC324F18EC325F190C326F191C327F1CE
:1030600001011D6BF9EC1CF070EC1CF0880E046F74
:10307000130E056F000E066F000E076FB8EC1BF005
:10308000000E046F040E056F000E066F000E076F32
:10309000C3EC1BF00101E80E046F800E056F000EFB
:1030A000066F000E076FE2EC1BF00A0E0C6E00C1FB
:1030B0000BF032EC07F00B0E0C6E01C10BF032EC92
:1030C00007F00C0E0C6E02C10BF032EC07F00D0E87
:1030D0000C6E03C10BF032EC07F004017A0E826F24
:1030E00002EC0AF004012C0E826F02EC0AF00401DB
:1030F000360E826F02EC0AF004012C0E826F02EC95
:103100000AF032EC17F04BEF12F087C31EF188C3C0
:103110001FF189C320F18AC321F18BC322F18CC333
:1031200023F18DC324F18FC325F190C326F191C300
:1031300027F10101F9EC1CF070EC1CF0000E046F9B
:10314000120E056F000E066F000E076FC3EC1BF02A
:1031500001010A0E046F000E056F000E066F000ECF
:10316000076FE2EC1BF0120E0C6E00C10BF032EC9C
:1031700007F0130E0C6E01C10BF032EC07F0140EC9
:103180000C6E02C10BF032EC07F0150E0C6E03C191
:103190000BF032EC07F004017A0E826F02EC0AF0B9
:1031A00004012C0E826F02EC0AF00401370E826FCC
:1031B00002EC0AF004012C0E826F02EC0AF0B6EC6D
:1031C00016F04BEF12F087C31EF188C31FF189C3BD
:1031D00020F18AC321F18BC322F18CC323F18DC36B
:1031E00024F18EC325F190C326F191C327F101018B
:1031F0001D6BF9EC1CF070EC1CF0880E046F130EC4
:10320000056F000E066F000E076FB8EC1BF0000E86
:10321000046F040E056F000E066F000E076FC3ECFF
:103220001BF00101E80E046F800E056F000E066FA3
:10323000000E076FE2EC1BF0060E0C6E00C10BF0E7
:1032400032EC07F0070E0C6E01C10BF032EC07F008
:10325000080E0C6E02C10BF032EC07F0090E0C6E7A
:1032600003C10BF032EC07F004017A0E826F02EC1E
:103270000AF004012C0E826F02EC0AF00401380EF1
:10328000826F02EC0AF004012C0E826F02EC0AF04D
:1032900048EC17F04BEF12F081A80AEF1AF007A8DC
:1032A000C3EF19F00101800E006F1A0E016F060EB8
:1032B000026F000E036F3EC104F13FC105F140C132
:1032C00006F141C107F1B4EC1BF003BF0AEF1AF09D
:1032D00074EC1AF03EC100F13FC101F140C102F1AE
:1032E00041C103F10782C1EC1AF00CC104F10DC118
:1032F00005F10EC106F10FC107F1F80E006FCD0EFA
:10330000016F660E026F030E036FB4EC1BF00E0E1E
:103310000C6E00C10BF032EC07F00F0E0C6E01C109
:103320000BF032EC07F0100E0C6E02C10BF032EC19
:1033300007F0110E0C6E03C10BF032EC07F007849E
:103340000101ABEC1CF04AC100F14BC101F1079443
:103350000A0E0C6E00C10BF032EC07F00B0E0C6E77
:1033600001C10BF032EC07F00C0E0C6E02C10BF039
:1033700032EC07F00D0E0C6E03C10BF032EC07F0CF
:1033800007980AEF1AF007AA0AEF1AF0078401015A
:10339000ABEC1CF04AC100F14BC101F10794060EE1
:1033A0000C6E00C10BF032EC07F0070E0C6E01C181
:1033B0000BF032EC07F0080E0C6E02C10BF032EC91
:1033C00007F0090E0C6E03C10BF032EC07F0078416
:1033D00055C100F156C101F157C102F158C103F1C5
:1033E0000794120E0C6E00C10BF032EC07F0130EB6
:1033F0000C6E01C10BF032EC07F0140E0C6E02C122
:103400000BF032EC07F0150E0C6E03C10BF032EC32
:1034100007F0079A0401805181197F0B0BE09EA8E9
:1034200009D014EE00F081517F0BE126E750812B8B
:103430000F01AD6E05012951010A13E081AA31EF98
:103440001AF005012951000A0AE00EB831EF1AF00E
:1034500005012A6731EF1AF00EB831EF1AF097EF35
:1034600022F081B846EF1AF0C8EC1DF00501295191
:10347000020A02E046EF1AF0562F46EF1AF055C541
:1034800056F50501010E2A6F3C0E2B6F70EF09F007
:103490000CC100F10DC101F10EC102F10FC103F128
:1034A000000E046F000E056F010E066F000E076F11
:1034B000E2EC1BF01DA173EF1AF01451D8B473EFB6
:1034C0001AF00CC100F10DC101F10EC102F10FC1E2
:1034D00003F1000E046F000E056F0A0E066F000E5A
:1034E000076FE2EC1BF0120001010C6B0D6B0E6B11
:1034F0000F6B12001EC182F40401300E822702EC11
:103500000AF01FC182F40401300E822702EC0AF097
:1035100020C182F40401300E822702EC0AF021C19E
:1035200082F40401300E822702EC0AF022C182F4F8
:103530000401300E822702EC0AF023C182F4040158
:10354000300E822702EC0AF024C182F40401300E0E
:10355000822702EC0AF025C182F40401300E822792
:1035600002EC0AF026C182F40401300E822702EC3C
:103570000AF027C182F40401300E822702EC0AF01F
:1035800012000101005305E1015303E1025301E17F
:10359000002B84EC1BF0ABEC1CF02C51006F2D5178
:1035A000016F420E046F4B0E056F000E066F000E8A
:1035B000076FC3EC1BF000C104F101C105F102C1AA
:1035C00006F103C107F10CC100F10DC101F10EC1FB
:1035D00002F10FC103F107B2F2EF1AF0B8EC1BF0E1
:1035E000F4EF1AF0B4EC1BF000C10CF101C10DF1C5
:1035F00002C10EF103C10FF11200ABEC1CF04CC183
:1036000000F14DC101F1060E48EC07F0E8CF04F1DE
:10361000070E48EC07F0E8CF05F1080E48EC07F07C
:10362000E8CF06F1090E48EC07F0E8CF07F1B4EC5B
:103630001BF000C118F101C119F102C11AF103C157
:103640001BF1290E046F000E056F000E066F000EB1
:10365000076FC3EC1BF0EE0E046F430E056F000EF8
:10366000066F000E076FB8EC1BF018C104F119C10A
:1036700005F11AC106F11BC107F1C3EC1BF000C133
:1036800010F101C111F102C112F103C113F1120EC7
:1036900048EC07F0E8CF04F1130E48EC07F0E8CF50
:1036A00005F1140E48EC07F0E8CF06F1150E48ECD2
:1036B00007F0E8CF07F10D0E006F000E016F000E4E
:1036C000026F000E036FC3EC1BF0180E046F000EA8
:1036D000056F000E066F000E076FE2EC1BF010C1C5
:1036E00004F111C105F112C106F113C107F1B8ECE3
:1036F0001BF06A0E046F2A0E056F000E066F000E97
:10370000076FB4EC1BF01200BF0EFA6E200E2D6F87
:103710002C6BD8900037013702370337D8B095EFBC
:103720001BF02D2F8AEF1BF02C072D070353D8B465
:1037300012000331070B8009326F03390F0B010FA1
:103740002C6F80EC5FF0336F2C0580EC5FF0335D05
:10375000335F2C6B3233D8B02C272C3332A9AAEF2D
:103760001BF033512C271200D0EC1CF0D8B0120003
:1037700003510719286F93EC1CF0D89007510319D7
:1037800028AF800F1200286BB7EC1CF0D8A0CDEC4E
:103790001CF0D8B01200A2EC1CF0ABEC1CF01F0E19
:1037A000296FE3EC1CF00B35D8B093EC1CF0D8A0DB
:1037B0000335D8B01200292FD1EF1BF028B1BAEC95
:1037C0001CF01200286B04510511061107110008A6
:1037D000D8A0B7EC1CF0D8A0CDEC1CF0D8B01200EB
:1037E000086B096B0A6B0B6BE3EC1CF01F0E296F67
:1037F000E3EC1CF007510B5DD8A40BEF1CF0065155
:103800000A5DD8A40BEF1CF00551095DD8A40BEF9D
:103810001CF00451085DD8A01EEF1CF00451085F95
:103820000551D8A0053D095F0651D8A0063D0A5FA5
:103830000751D8A0073D0B5FD8900081292FF8EFE2
:103840001BF028B1BAEC1CF0286BB7EC1CF0D89038
:10385000E7EC1CF007510B5DD8A43BEF1CF00651C0
:103860000A5DD8A43BEF1CF00551095DD8A43BEFDD
:103870001CF00451085DD8A04AEF1CF0003F4AEF4D
:103880001CF0013F4AEF1CF0023F4AEF1CF0032BF3
:10389000D8B4120028B1BAEC1CF012000101286B58
:1038A000B7EC1CF0D8B01200ECEC1CF0200E296F25
:1038B000003701370237033711EE27F00A0E2A6F5F
:1038C000E7360A0EE75CD8B0E76EE5522A2F60EFC4
:1038D0001CF0292F58EF1CF028B11D81D890120040
:1038E00001010A0E286F200E296F11EE1DF02851DC
:1038F0002A6F0A0ED890E652D8B0E726E7322A2F70
:103900007BEF1CF00333023301330033292F75EFB3
:103910001CF0E750FF0FD8A00335D8B012001DB13E
:10392000BAEC1CF01200045100270551D8B0053D37
:1039300001270651D8B0063D02270751D8B0073DF0
:10394000032712000051086F0151096F02510A6FDD
:1039500003510B6F12000101006B016B026B036BD3
:1039600012000101046B056B066B076B1200033537
:10397000D8A012000351800B001F011F021F031F5C
:10398000003FCAEF1CF0013FCAEF1CF0023FCAEF34
:103990001CF0032B282B032512000735D8A012009A
:1039A0000751800B041F051F061F071F043FE0EF90
:1039B0001CF0053FE0EF1CF0063FE0EF1CF0072B8A
:1039C000282B072512000037013702370337083745
:1039D00009370A370B37120001011D6B1E6B1F6B75
:1039E000206B216B226B236B246B256B266B276B63
:1039F00012001E510F0B1E6F1F510F0B1F6F205116
:103A00000F0B206F21510F0B216F22510F0B226FD3
:103A100023510F0B236F24510F0B246F25510F0BD4
:103A2000256F26510F0B266F27510F0B276F1200A2
:103A30008984000EC76E220EC66E9E96C69E000E2C
:103A4000C96EFF0E9EB602D0E82EFCD79E96C69E8B
:103A5000000EC96EFF0E9EB602D0E82EFCD7C9CF6D
:103A6000A5F59E96C69E000EC96EFF0E9EB602D0AC
:103A7000E82EFCD7C9CFA6F59E96C69E000EC96E4D
:103A8000FF0E9EB602D0E82EFCD7C9CFA7F59E96B2
:103A9000C69E000EC96EFF0E9EB602D0E82EFCD761
:103AA000C9CFA8F59E96C69E000EC96EFF0E9EB6A3
:103AB00002D0E82EFCD7C9CFA9F59E96C69E000E6F
:103AC000C96EFF0E9EB602D0E82EFCD7C9CFAAF56C
:103AD0009E96C69E000EC96EFF0E9EB602D0E82EC0
:103AE000FCD7C9CFABF5899474EC1FF01200898420
:103AF000000EC76E220EC66E9E96C69E800EC96EC2
:103B0000FF0E9EB602D0E82EFCD79E96C69EA5C597
:103B1000C9FFFF0E9EB602D0E82EFCD79E96C69E29
:103B2000A6C5C9FFFF0E9EB602D0E82EFCD79E9612
:103B3000C69EA7C5C9FFFF0E9EB602D0E82EFCD7D1
:103B40009E96C69EA8C5C9FFFF0E9EB602D0E82E5F
:103B5000FCD79E96C69EA9C5C9FFFF0E9EB602D091
:103B6000E82EFCD79E96C69EAAC5C9FFFF0E9EB63C
:103B700002D0E82EFCD79E96C69EABC5C9FFFF0EAD
:103B80009EB602D0E82EFCD7899474EC1FF0120088
:103B90008984000EC76E220EC66E9E96C69E070EC4
:103BA000C96EFF0E9EB602D0E82EFCD79E96C69E2A
:103BB000000EC96EFF0E9EB602D0E82EFCD7C9CF0C
:103BC000A5F59E96C69E000EC96EFF0E9EB602D04B
:103BD000E82EFCD7C9CFA6F59E96C69E000EC96EEC
:103BE000FF0E9EB602D0E82EFCD7C9CFA7F59E9651
:103BF000C69E000EC96EFF0E9EB602D0E82EFCD700
:103C0000C9CFA8F5899474EC1FF08984000EC76EA3
:103C1000220EC66E9E96C69E0F0EC96EFF0E9EB6F3
:103C200002D0E82EFCD79E96C69E000EC96EFF0EEF
:103C30009EB602D0E82EFCD7C9CFADF5899474ECBE
:103C40001FF012008984000EC76E220EC66E9E966B
:103C5000C69E870EC96EFF0E9EB602D0E82EFCD718
:103C60009E96C69EA5C5C9FFFF0E9EB602D0E82E41
:103C7000FCD79E96C69EA6C5C9FFFF0E9EB602D073
:103C8000E82EFCD79E96C69EA7C5C9FFFF0E9EB61E
:103C900002D0E82EFCD79E96C69EA8C5C9FFFF0E8F
:103CA0009EB602D0E82EFCD7899474EC1FF089846C
:103CB0009E96C69E8F0EC96EFF0E9EB602D0E82E4F
:103CC000FCD79E96C69EADC5C9FFFF0E9EB602D01C
:103CD000E82EFCD7899474EC1FF012008984000E42
:103CE000C76E220EC66E9E96C69E870EC96EFF0ECA
:103CF0009EB602D0E82EFCD79E96C69E000EC96ED8
:103D0000FF0E9EB602D0E82EFCD79E96C69E800E71
:103D1000C96EFF0E9EB602D0E82EFCD79E96C69EB8
:103D2000800EC96EFF0E9EB602D0E82EFCD79E967E
:103D3000C69E800EC96EFF0E9EB602D0E82EFCD73E
:103D4000899474EC1FF089849E96C69E8F0EC96E6E
:103D5000FF0E9EB602D0E82EFCD79E96C69E010EA0
:103D6000C96EFF0E9EB602D0E82EFCD7899474EC83
:103D70001FF012008984000EC76E220EC66E9E963A
:103D8000C69E870EC96EFF0E9EB602D0E82EFCD7E7
:103D90009E96C69E000EC96EFF0E9EB602D0E82EFD
:103DA000FCD79E96C69E000EC96EFF0E9EB602D030
:103DB000E82EFCD79E96C69E800EC96EFF0E9EB65C
:103DC00002D0E82EFCD79E96C69E800EC96EFF0ECE
:103DD0009EB602D0E82EFCD7899474EC1FF089843B
:103DE0009E96C69E8F0EC96EFF0E9EB602D0E82E1E
:103DF000FCD79E96C69E010EC96EFF0E9EB602D0DF
:103E0000E82EFCD7899474EC1FF012008984000E10
:103E1000C76E220EC66E9E96C69E8F0EC96EFF0E90
:103E20009EB602D0E82EFCD774EC1FF09E96C69E7C
:103E3000810EC96EFF0E9EB602D0E82EFCD7899483
:103E400074EC1FF08984000EC76E220EC66E9E961B
:103E5000C69E8F0EC96EFF0E9EB602D0E82EFCD70E
:103E600074EC1FF09E96C69E010EC96EFF0E9EB6A4
:103E700002D0E82EFCD7899474EC1FF089849E96BA
:103E8000C69E910EC96EFF0E9EB602D0E82EFCD7DC
:103E900074EC1FF09E96C69EA50EC96EFF0E9EB6D0
:103EA00002D0E82EFCD7899474EC1FF012008984AC
:103EB000000EC76E220EC66E9E96C69E910EC96EED
:103EC000FF0E9EB602D0E82EFCD774EC1FF09E9633
:103ED000C69E000EC96EFF0E9EB602D0E82EFCD71D
:103EE000899474EC1FF01200050EE82EFED7120024
:103EF000200EC66E0501256B266B276B286B899AF1
:103F0000400EC76E200EC66E9E96C69E030EC96EEC
:103F1000FF0E9EB602D0E82EFCD79E96C69E27C501
:103F2000C9FFFF0E9EB602D0E82EFCD79E96C69E15
:103F300026C5C9FFFF0E9EB602D0E82EFCD79E967E
:103F4000C69E25C5C9FFFF0E9EB602D0E82EFCD73F
:103F50009E96C69EC952FF0E9EB602D0E82EFCD792
:103F6000898AC950FF0A02E1BFEF1FF0100E252712
:103F7000E86A2623E86A272327A97FEF1FF0220E8D
:103F8000C66E1200899A400EC76E200EC66E9E96AF
:103F9000C69E060EC96EFF0E9EB602D0E82EFCD756
:103FA000898A899A9E96C69EC70EC96EFF0E9EB6D6
:103FB00002D0E82EFCD7898A899A9E96C69E050E65
:103FC000C96EFF0E9EB602D0E82EFCD79E96C69E06
:103FD000C952FF0E9EB602D0E82EFCD7C9B0E6EF5C
:103FE0001FF0898A0501256B266B276B286B120051
:103FF0000501FE0E2D6F0501000E2D6F18EC1DF052
:10400000A5C52EF5A6C52FF5A7C530F5A8C531F570
:10401000A9C532F5AAC533F5ABC534F50784A9C1E6
:1040200059F1AAC15AF1ABC15BF1ACC15CF13EC11F
:1040300042F13FC143F140C144F141C145F14AC1A0
:104040004CF14BC14DF1079475EC12F000C135F500
:1040500001C136F502C137F503C138F505015767CF
:1040600039EF20F0586739EF20F0596739EF20F029
:104070005A673DEF20F04BEF20F057C504F158C5CB
:1040800005F159C506F15AC507F10101B4EC1BF061
:1040900003BFB9EF20F04CC139F54DC13AF5AFC5BA
:1040A0003BF5B0C53CF50501100E2C6F899A400E0A
:1040B000C76E200EC66E9E96C69E060EC96EFF0E79
:1040C0009EB602D0E82EFCD7898A899A9E96C69E13
:1040D000020EC96EFF0E9EB602D0E82EFCD79E9649
:1040E000C69E27C5C9FFFF0E9EB602D0E82EFCD79C
:1040F0009E96C69E26C5C9FFFF0E9EB602D0E82E2C
:10410000FCD79E96C69E25C5C9FFFF0E9EB602D05F
:10411000E82EFCD725EE2DF02C2F02D09BEF20F0BF
:104120009E96C69EDECFC9FFFF0E9EB602D0E82E39
:10413000FCD78CEF20F0898A899A9E96C69E050E40
:10414000C96EFF0E9EB602D0E82EFCD79E96C69E84
:10415000C952FF0E9EB602D0E82EFCD7C9B0A6EF1A
:1041600020F0898A0501100E2527E86A2623E86ACF
:104170002723120019C502F51AC503F525EE5FF0D5
:1041800005012C6B16EE00F005010251E1260351EA
:10419000D8B00329E226E7CFE8FF2C0A06E12CC5B8
:1041A000DEFF05012C6BDDEF20F0E7CFE8FF2A0AE8
:1041B0000CE0E7CFDEFF05012C2B0501032B023FAE
:1041C0000307030E0317C2EF20F005012D6B2E6BC2
:1041D0002F6B306B316B326B336B346B356B366BF3
:1041E000376B386B396B3A6B3B6B3C6B3D6B3E6BA3
:1041F0003F6B406B416B426B436B446B456B466B53
:10420000476B486B496B4A6B4B6B4C6BDDCFE8FFE0
:1042100005012C5105E0DDCFE8FF2C2F0BEF21F03D
:104220000501DDCF2CF52C5105E0DDCFE8FF2C2F6B
:1042300015EF21F00501DDCF2CF52C5105E0DDCF88
:10424000E8FF2C2F1FEF21F011EE27F00101ECEC1D
:104250001CF00501DDCF2CF52C5105E0DDCFE5FF8D
:104260002C2F2EEF21F00101F9EC1CF070EC1CF06A
:1042700000C12EF501C12FF502C130F50501DDCFDA
:104280002CF52C5105E0DDCFE8FF2C2F43EF21F07A
:104290000501DDCF2CF52C5105E0DDCFE8FF2C2FFB
:1042A0004DEF21F00501DDCF2CF52C5107E0DDCFDE
:1042B000E8FFE8A82D852C2F57EF21F011EE27F00D
:1042C0000101ECEC1CF00501DDCF2CF52C5114E0C4
:1042D000DDCFE5FFDDCFE5FFDDCFE5FFDDCFE5FF9E
:1042E000DDCFE8FFDDCFE5FFDDCFE5FFDDCFE5FF8B
:1042F000DDCFE5FFDDCFE5FF0101F9EC1CF070EC4F
:104300001CF000C138F501C139F502C13AF503C10D
:104310003BF50501DDCF2CF52C5107E0DDCFE8FFA3
:10432000E8A82D832C2F8EEF21F011EE27F001014C
:10433000ECEC1CF00501DDCF2CF52C5105E0DDCFB8
:10434000E5FF2C2F9FEF21F0010122C123F121C1B4
:1043500022F120C121F11FC120F1F9EC1CF070EC19
:104360001CF000C134F501C135F502C136F503C1B9
:1043700037F50501DDCF2CF52C5107E0DDCFE8FF47
:104380002C2FBEEF21F0E8B02D8711EE27F00101B0
:10439000ECEC1CF0DDCFE8FFDDCFE8FFDDCFE8FF80
:1043A000DDCFE8FFDDCFE8FFDDCFE5FFDDCFE5FFC7
:1043B000DDCFE5FFDDCFE5FFDDCFE5FFDDCFE5FFBD
:1043C000F9EC1CF070EC1CF000C131F501C132F5C4
:1043D00002C133F5078455C159F156C15AF157C18D
:1043E0005BF158C15CF13EC142F13FC143F140C1B4
:1043F00044F141C145F14AC14CF14BC14DF1079423
:1044000075EC12F000C13CF501C13DF502C13EF56D
:1044100003C13FF5120021C500F122C501F123C5FA
:1044200002F124C503F1899A400EC76E200EC66EB4
:104430009E96C69E0B0EC96EFF0E9EB602D0E82E4B
:10444000FCD79E96C69E02C1C9FFFF0E9EB602D043
:10445000E82EFCD79E96C69E01C1C9FFFF0E9EB6F0
:1044600002D0E82EFCD79E96C69E00C1C9FFFF0E63
:104470009EB602D0E82EFCD79E96C69EC952FF0E6D
:104480009EB602D0E82EFCD725EE2DF00501100EC9
:104490002C6F9E96C69EC952FF0E9EB602D0E82E85
:1044A000FCD7C9CFDEFF2C2F49EF22F0898A1200FA
:1044B000899A400EC76E200EC66E9E96C69E900EBE
:1044C000C96EFF0E9EB602D0E82EFCD79E96C69E01
:1044D000000EC96EFF0E9EB602D0E82EFCD79E9647
:1044E000C69E000EC96EFF0E9EB602D0E82EFCD707
:1044F0009E96C69E000EC96EFF0E9EB602D0E82E96
:10450000FCD79E96C69EC952FF0E9EB602D0E82EDC
:10451000FCD7C9CF2DF59E96C69EC952FF0E9EB6FA
:1045200002D0E82EFCD7C9CF2EF5898A1200C8EC3C
:104530001DF0F29CF29E8B948A86899CC69AC2904A
:104540008A94898A9482948C720ED36ED3A4FED7F7
:1045500089968A909390FF0EE8CF00F0E82EFED760
:10456000002EFCD78150F294F29A9E909D909E92DC
:104570009D92F298F292F290F286F28E0300FF0082
:10BF0000E844F926000C160C2B0C3F0C520C640C68
:10BF1000760C860C960CA50CB30CC10CCF0CDC0C6B
:06BF2000E80CF40C000C1B
:00000001FF
